:030000000219FDE5
:03000B000200AA46
:03002B0002015679
:03005B000202ECB2
:030073000202D2B4
:1000800002030406080C10182030406080040608A3
:100090000C10182030406080A0C000070F1F3F0DDB
:1000A0000D0403060D0503030202C2AFC0D0C0E079
:1000B000206217E5256002E473E525F4F58A758B67
:1000C00000D262D0E0D0D0D2AF3285268AC262E5BB
:1000D00026F46035306803207210758B00D0E0D0B4
:1000E000D0D295D293D297D2AF32D295D293D29723
:1000F000206E0C206609740CD5E0FDE57E429075FB
:100100008B00D0E0D0D0D2AF32758A00C28DD262DF
:1001100001FF01B9306805206602C29501B9306857
:1001200005206602C29701B9306805206602C293B5
:1001300001B9C294306805206602C29501B9C29621
:10014000306805206602C29701B9C2923068052066
:100150006602C29301B9C2AFC2AD53E6EFC0D0C0D0
:10016000E0D2D3D2AFC2CEE52A6007207449152A67
:1001700021B77800790020742EE580307E01F430BC
:10018000E50278FF53DACF207E0343DA20307E0386
:1001900043DA10C2D8C271E580307E01F430E50246
:1001A00079FFC3E89970CB306103752A402074034E
:1001B000752A40885FD27020740DE52B6004152BE2
:1001C00021C743DA01C2D820700221DAA85F20617A
:1001D00002C27020740221D888227882B604038576
:1001E0002224C3E52594404002D26420CF0AD0E007
:1001F000D0D043E610D2AD32C2CF053A7802E52A1C
:100200006005307402152AC3E55F940140057562EC
:10021000004124756300756C00E5622401F56250AD
:10022000037562FF7982B7020D306D1DC3E522941C
:10023000324016854D227982B7030E306D0BC3E52F
:100240002294324004798E8722C3E52395226008E8
:100250004004152341580523D8CA056CE56C70028B
:10026000156CD56D63756D017805C3E56C956E40B1
:1002700057C3E56C956F50087801756D0302028CC9
:10028000C3E56C957050057801756D01C3E5659502
:1002900024401E7982B7040241BD206D1485246577
:1002A000E56C046003856E6C756D0175233C02027C
:1002B000C8E5652850057565FF41BDF565E5650430
:1002C00070067563FF756CFFD0E0D0D043E610D2A6
:1002D000AD32C2AFC0D053E67FC260759100855683
:1002E00094855795759104D0D0D2AF32C2AF53E602
:1002F000EFC2ADC0D0C0E0C0F0D2D3D2AFA8FBA94E
:10030000FCC2D8307102615353DACF207E0343DA46
:1003100010307E0343DA20D271E580307E01F42074
:10032000E502612A88278928A13853DACF207E0385
:1003300043DA20307E0343DA10C2D8C2713074022F
:10034000A1247800E580307E01F430E502A1248804
:100350005FA10C53DACF207E0343DA20307E0343C3
:10036000DA10C271206102812C53DACF207E034360
:10037000DA10307E0343DA20C2D8D271885A895B02
:10038000C3E89558F8E99559F97B007E087A00C3CF
:10039000E8948CE994005005755E00811E882178F0
:1003A000A2E6A8216055C3E894C8E994005008E487
:1003B000D2E4FB7A0A61F9C3E89468E99401500831
:1003C000E4D2E3FB7A0F61F9C3E894D0E9940250D8
:1003D00008E4D2E2FB7A1E61F9C3E894A0E994052F
:1003E0005008E4D2E1FB7A3C61F9C3E89498E994BF
:1003F000085008E4D2E0FB7A787E00C3E8955CFC04
:10040000E9955DFD30E70AECF42401FCEDF43400DD
:10041000FD755E00C3EC9AED9E5003755E01885C2D
:10042000895D855A58855B597802A10CC3E89527E8
:10043000F8E99528F9307C0281F0307B0281F030B8
:100440007A0281E9207502814FE9FDE8FC816EE9BD
:10045000C313F9E813F830790281E9E9C313F9E825
:1004600013F830780281E9E9C313FDE813FC206139
:0F0470002CC3EC941CED940240028185ED701EAC
:10047F00C3EC94C850180529E52970021529C3E566
:10048F0029940A5002A124755F00D270A124E52996
:10049F00600215297400207F037896E624FAFEE4A3
:1004AF003400FFC3EC9EFCED9FFD500678007900F1
:1004BF0081F0C3EC94FFED9400400678FF79008142
:1004CF00F0EC8575F0A4C5F0A2F733F8790040037E
:1004DF0002050C78FF790002050CE9C313F9E81344
:1004EF00F8307C0EE9600278FFC3E81338F8E43483
:1004FF0000F9C3E894FFE99400400278FF885FD2C7
:10050F0070206102A124741FF4552F4BF52FC27474
:10051F00EB7002D274752A40307403752A0A306169
:10052F0002A13820740353DAFE207403752B20D0F8
:10053F00F0D0E0D0D0D2AD43E61032790102056899
:10054F007903020568790A020568791E0205687940
:10055F006402056879C80205687817E4D5E0FDD80C
:10056F00FAD9F6227A147B7802058F7A107B8C02E7
:10057F00058F7A0D7BB402058F7A0B7BC802058F2E
:10058F007902B27DE4C296D5E0FDC297D5E0FDD2E7
:10059F0097D5E0FDD296D5E0FDC295E576D5E0FD85
:1005AF00D2957496D5E0FDD9D9EAF8D5E0FDD8FB00
:1005BF00DBCEC29622C37C007D0075F00005F0EA09
:1005CF0033FAEB33FB50F6EB13FBEA13FAC3E9FFF5
:1005DF00E8FEE89AF8E99BF95004EFF9EEF8B3EC6E
:1005EF0033FCED33FDD5F0DFEDF9ECF822E889F0BF
:1005FF008A20D2D4F8A9F07B0030F70B7BFFF424CC
:10060F0001F8E9F43400F9E88520F0A4ADF0F8E939
:10061F008520F0A4AFF0FEED2EF974003FFA7C04B4
:10062F00C3EA13FAE913F9E813F8DCF48BF030F7A7
:10063F000AE8F42401F8E9F43400F9E889F0C2D4A7
:10064F00F8A9F0227882B604030206F2C3E55F949C
:10065F0019401EE52D54067018206D3678057994D3
:10066F00E7146007780A1460027812C3E5419840D6
:10067F001F306D09856765756CFF756D01852224C7
:10068F00E4F545F546F547F548F549C26D0206F222
:10069F00D26D7994E7147013E523F43333F913F81B
:1006AF00E9540104F9E854FE0206E6E71414701445
:1006BF00E523F4333333F913F8E9540304F9E85419
:1006CF00FC0206EEE523F433333333F913F8E95420
:1006DF00070404F9E854F8C39440F8E99400F98842
:1006EF0045894622C3E54113F9E54013F8C3E545B3
:1006FF0098F8E54699F9500CC3E89480E994FF40C7
:10070F001602072AC3E8947FE99400500302072AD0
:10071F00787F790002072A788079FF884A894B22EF
:10072F00E54A2547F8E54B3548F9854B20E4300776
:10073F0001F43549FA30E709C3EA94F0401502078E
:10074F0068C3EA940F500302076878FF79FF7A0FA6
:10075F00020768780079007AF0C3E5249564500A9F
:10076F00C374019524500B020786E54B20E70E0258
:10077F000786E54B30E706884789488A492278A4DF
:10078F00E6FAC3E54A33F8E54B33F9B1FCE930E754
:10079F000BC3E89480E994FF4013E1C0C3E8947F52
:1007AF00E994005002E1C0787F7900E1C078807948
:1007BF00FFE820E715C3E52398F84009C3E8940143
:1007CF0040030207E778010207E7E8F42401252335
:1007DF00F840030207E778FF884C2278A5E6FAA8CD
:1007EF0048A949B1FCE930E70CC3E89401E994FF4B
:1007FF00401602081BC3E894FFE994005003020857
:10080F001B78FF790002081B780179FFE920E715B3
:10081F00C3E54C98F84009C3E8940140030208422D
:10082F007801020842E8F42401254CF8400302083D
:10083F004278FF88242278FFC26420693D206A1223
:10084F00D264C3E541940A4009C3E52594405002A0
:10085F00C26479A1E76023E541601F74FF8541F011
:0E086F00848539F0306A0375F005A4F8C5F0F1
:10087D00600278FFC3E895675002A867886622C3B7
:10088D00E5409440E5419401E566500314019D0453
:10089D006002F566227883E6F520120F3B75E8902D
:1008AD0012054A75E890E5E820ECFBA8BDA9BE123B
:1008BD000FD5757155757200C3740013FD745560B5
:1008CD006613FC74552CFC74003DFDECFAEDFBC376
:1008DD00E89AE99B4014E5712455F571E5723400F1
:1008ED00F572EA2CFAEB3DFB80E5AE71AF72C3E514
:1008FD007213F9E57113F8C3E913F9E813F87A03E4
:10090D00C3E913F9E813F8DAF7AA201A700975711B
:10091D00007572000209341AEA6008EE28FEEF39FC
:10092D00FFDAF88E718F722275E890227883E6FFD8
:10093D00E5E820ECF7A8BDA9BE0573C3E5739408DF
:10094D004052757300E9FA79A0E76044EA7007E553
:10095D0074601B02096FC3E895746010E57450064E
:10096D00600C1402097B0460F902097BE574F574CF
:10097D00C3946D401B7564C0C394044013756480AB
:10098D00C39404400B756440C39404400375640024
:10099D0075BB0822EFC39401601F7455601BC3E83B
:1009AD0094FFE994035012C3E89571E995725009CB
:1009BD00E564600C15640209CDE564F4600205641C
:1009CD00A864C3E524985002A824C3E89565400A9D
:1009DD00A865E565F4600385656488258826E5735B
:1009ED00B4070375BB1022743279A687F0A4C5F045
:1009FD00A2F733F8C3E895644002A86488228824DE
:100A0D00882588268867227540007541F022C2AF7F
:100A1D0075C820A8CCA9CDAA3A30CF010A75C82433
:100A2D00D2AFAB3BAC3C883B893CC3E89BF8E99C1F
:100A3D00206908F93067026130418DAD3D8A3DF97D
:100A4D00EA9DFA600478FF79FFAE3EAF3F8B3E8C96
:100A5D003FC3EC9FFCC3E99CF542A83BA93CC3E80E
:100A6D009EF8E99FF9C3E54113FBE54013FAE82A27
:100A7D00F540E93BF54150067540FF7541FF41D703
:100A8D00AA40AB41AC40AD417E047F02C3EB940460
:100A9D0040021E1FC3EB940840021E1FC3ED13FD41
:100AAD00EC13FCDEF7C3EA9CFAEB9DFBEF6009C388
:100ABD00E913F9E813F8DFF7EA28FAEB39FB8A4076
:100ACD008B4150067BFF8B408B41C3EB9402500250
:100ADD00D2673069047F0361027892E6FFC3E53780
:100AED00948240110FC3E53794A040010FC3EF94DA
:100AFD000640027F057E05E541C4540FF9E541C46A
:100B0D0054F0F8E540C4540F28F8C3E89EFAE99470
:100B1D0000FB4009C3EA9402EB940050047A02E40E
:100B2D00FB617CAA40AB41EBC4FEEAC4540F4EFC02
:100B3D00C3EA9CFAEB9400FBC3E813C313F8EA284D
:100B4D00FAEB3400FB8A408B41C3EB94024002C2A6
:100B5D00677805EBC4FE7B00EAC4540F4EFAC3EA76
:100B6D0098FA4005C3940250027A027892E6FF305B
:100B7D006002617C855256855357D26043E680C32F
:100B8D00E49AF8E49BF93067028116E8FAE9FBD3A1
:100B9D00E913FDE813FC88528953C3EF94036038C1
:100BAD00EF20E00DE82CF8E93DF9ECFAEDFB020B36
:100BBD00D1E828F8E939F9C3E82402F8E93400F955
:100BCD007AFE7BFFC3EF9403400E8A548B55884EFB
:100BDD00894F8C508D51814A885489558A4E8B4F3F
:100BED008C508D51306920C3E53394034019E54293
:100BFD00A2E713F8E555F4240138400B20E70875FA
:100C0D0054FFF42401F555814AE8FAD3E813FC8822
:100C1D0052C3EF94036020EF20E007E82CF8ECFAC4
:100C2D008136E8282402F87AFEC3EF940340088A3F
:100C3D0054884E8C50814A88548A4E8C50E56BC333
:100C4D00335002646BF56B3060028154753402D2FF
:100C5D006043E680E52D54066026A840A941C3E90E
:0F0C6D0013F9E813F8C2AF53E67F759100C3E4A3
:100C7C0098F594E499F595759104D26043E680D289
:100C8C00AF22D265754400752000306B037520408F
:100C9C00020CADD265754400752040306B03752095
:100CAC0000D2AF7801206722E52D54066002C265A0
:100CBC00C3E54194054013780294054008780394E9
:100CCC000540027806306902780A206019E5446014
:100CDC001530690AC3E53394034003D53406D2AF0B
:100CEC00D26CA17E915CD2AF0000C2AF206726E52A
:100CFC0041C3FB940F40027B0FEB2405307301239F
:100D0C00306A02742820620123F93069027982E585
:100D1C008BC39940B50544E59B5440B52002A168AE
:100D2C0030690A08C3E8940A40010881D62065029C
:100D3C0081ADC26553E67F759100306710759400E4
:100D4C007595FE759104D26043E68081ADAE40AFDF
:100D5C0041C3E49EF594E49FF595A14FC3E533940C
:100D6C0002500281AD30650281ADD802A17C81D6E2
:100D7C00C26C53E67F759100855494855595759199
:100D8C0004854E56854F57D26043E680D2AFE52D91
:100D9C0054066008206A020533020DB8306C0D2031
:100DAC006B0A2065071581158102160D227800301B
:100DBC0064053065027801E53775F007A4F9E5F0B4
:100DCC0028F5F0E9A2F013A2F113A2F213F537C340
:100DDC0094785003753778C3E53795384008D26658
:100DEC00D295D293D297306002A1F285505685519C
:100DFC0057D26043E68022207D11C2AF754302C2F8
:100E0C0096D294D2AF759F11020FD2C2AF75430226
:100E1C00C296D292D2AF759F11020FD2307243207C
:100E2C007D20C2AF75430390013E757E40D293C2C4
:100E3C0092306204C297C146D296D2AF759F13020C
:100E4C000FD2C2AF75430390013E757E40D295C25E
:100E5C0094306204C297C166D296D2AF759F1002CD
:100E6C000FD2207D17C2AF75430390011ED2933071
:100E7C006202C297D2AF759F13020FD2C2AF7543F5
:100E8C000390011ED295306202C297D2AF759F10AB
:100E9C00020FD2207D11C2AF754304C294D292D2FC
:100EAC00AF759F10020FD2C2AF754304C292D29499
:100EBC00D2AF759F13020FD2307243207D20C2AF88
:100ECC00754305900132757E10D297C2963062043C
:100EDC00C295C1E2D294D2AF759F11020FD2C2AFAC
:100EEC0075430590014A757E04D297C29630620410
:100EFC00C293E102D292D2AF759F11020FD2207D24
:100F0C0017C2AF754305900114D297306202C29597
:100F1C00D2AF759F11020FD2C2AF75430590012855
:100F2C00D2973062EBC293D2AF759F11020FD220D1
:100F3C007D11C2AF754306C292D296D2AF759F1384
:100F4C00020FD2C2AF754306C294D296D2AF759F30
:100F5C0010020FD2307242207D20C2AF7543019037
:100F6C00014A757E04D295C294306204C293E17E2C
:100F7C00D292D2AF759F10020FD2C2AF75430190BF
:100F8C000132757E10D293C292306204C295E19EFA
:100F9C00D294D2AF759F13E1D2207D16C2AF7543A8
:100FAC0001900128D295306202C293D2AF759F1086
:100FBC00E1D2C2AF754301900114D293306202C2E8
:100FCC0095D2AF759F13C26622900112757E00D226
:100FDC0095D293D297C294C292C296C26222788062
:100FEC0076070876070876010876040876FF0876F7
:100FFC00FF08760A087602087601087601788C7666
:10100C00010876000876B40876FF0876FF0876FFAC
:10101C000876030876FF0876010876FF087625081F
:10102C0076D00876780876C80876040876FF0876B5
:10103C000108760008767A08760A087601087601A7
:10104C000876000876FF227887E6FFC272BF03029B
:10105C00D2727888C27DE630E102D27DC27E788978
:0F106C00E630E102D27EC3EF94026008758E0178
:10107B00D273021085758E00C273227880E61490AD
:10108B0000809378A4F67881E6149000809378A57D
:10109B00F67886E61490008D9378A6F6789FE6F89E
:1010AB00700108C3E8941140027811E82828F56E06
:1010BB00256E256E28F56F256E2828F570789CE631
:1010CB007538FF75390CB402067538A075390AB43A
:1010DB00030675388275390578A3E61490009A9348
:1010EB00F569120FD522227896E6FA7897E6FB7807
:1010FB0088E6B40305C3EB940EFB307F047A007BC8
:10110B00FFC3EB9AFCC3948250027C827575000579
:10111B0075EC8575F0A4C3E5F0947D40F222D27F87
:10112B0011F21205597A007B007C1012054FE55F16
:10113B002AFA74003BFBDCF37C04C3EB13FBEA13CE
:10114B00FADCF7FEC27F11F222E5EF20E6037520F1
:10115B00000520903FFFE520146006901DFF1460F2
:10116B00009304600375EF1253D9BF7581C043FF21
:10117B008012054A75EF0243B203E5B3240420E75E
:10118B000DF521E5E320E0068521B343E301120FC2
:10119B00D57580FF75A40075F1B275D4DF7590A974
:1011AB0075A5FC75F2FE75D50175A60175E241E4D6
:1011BB00F8F6D8FD756B01120FEA12165578988662
:1011CB0076753001C2AF1205631205731205591201
:1011DB00057A120559120581120559121778120555
:1011EB006312056312055EC2AF78FA79FA30850790
:1011FB00D9FBD8F7021C001153118611F111F278AB
:10120B00988676120FD575885075891275C8247516
:10121B00910475D84075A82275B80275E690759B38
:10122B0080759D0075D10E75BC5875BB0875BA11CC
:10123B0075E88012054AD2AF1208A253DACF207E8E
:10124B000343DA20307E0343DA1043DA01C2D8C2FB
:10125B0071120563D2617B037A0CE55E70077A0C21
:10126B00DB030211F21205592070030211F2C27056
:10127B00E55FC3940240E1E52F541F856160F56182
:10128B00B560D5DAD5C26153DACF207E0343DA20BD
:10129B00307E0343DA10C2D8C27178A2E67008D24E
:1012AB0074E52F54E0F52FC27575290012055E30D9
:1012BB007409C3E529940A4002D27512054F7802CE
:1012CB003074027800C3E55F9840F0C2AF1205732B
:1012DB00120573120573D2AF120563754D0012051B
:1012EB004F788CE6C3940150030213BFE530C394CF
:1012FB000150030213BF207435C3E55F94FF500305
:10130B000213BFC2AF120588D2AF12055EC3E55FF1
:10131B00940150EFC2AF120573120554120573D22C
:10132B00AF12055EC3E55F94FF40E90217FD7F0531
:10133B00D27F11F212055EC2AFC27F11F2AE5FC354
:10134B00E55F947FD2AF407612054AC2AF12058893
:10135B00D2AFDFDC3129C3EE94057897F612056323
:10136B001216971217807F0AD27F11F212055EC2F6
:10137B00AFC27F11F2AE5FC3E55F947FD2AF50E691
:10138B0012054AC2AF120573120554120573D2AF80
:10139B00DFD63129EE24057896F6120563121697DF
:1013AB001217AF12055E11F2C3E55F94FF50026195
:1013BB00010217FDC3E55F954D4003855F4D120597
:1013CB005E78017988E7B403027805C3E55F98403E
:1013DB000241E9C2AF120588120588120588D2AF07
:1013EB00120563753000E4F531F5320531E531F462
:1013FB0070390532789AE6781914601278321460D5
:10140B000D787D14600878FA146003753200C3E51B
:10141B003298401715327531B478998676C2AF126F
:10142B000588D2AF7898867612055E120554E52AA8
:10143B00700530740221F278012074027806C3E53E
:10144B005F9840A712055EE52A70030211F2C2AF46
:10145B00120FD5E4F522F523F524F525F526F56ACB
:0E146B00D2AF7885E6C333F568E4F545F54663
:10147900F547F548F549F573F52CF52DF5377573ED
:101489000875BB1012054A120935E5E820ECFBA8DE
:10149900BDA9BEE97001F888741209397573087518
:1014A900BB107887E6FE760211537887EEF6C2AF55
:1014B9007564FF1209F4852264852265852266D246
:1014C900AF75220175240175250175260185636CA7
:1014D900756D017888E6B40307C27D307602D27D46
:1014E900D268D269753300120F3B120F60120A14C9
:1014F900120A1B120A14120A1B120A14021514C228
:10150900AF1153D2AF75730075BB08120C9F120649
:1015190053120DB9120E03120A1B120C8E306D03F1
:101529001206F320670312084530670312088C126C
:101539000DB9120E28120A1B120C9F306D031207E7
:101549002F120DB9120E9F120A1B120C8E306D0349
:1015590012078D120DB9120EC4120A1B120C9F30FC
:101569006D031207EA120DB9120F3B120A1B120979
:1015790035120C8E120DB9120F60120939120A1B9D
:1015890030692F206B2C85676485676585636C7569
:101599006D0179187A0CC3E533994009C269D26A99
:1015A9008A350215BBC3E55F940140030215140295
:1015B9001615306A1B206B18E535147004C26AA130
:1015C90008F535C3E55F94014003021514021615A9
:1015D900753600C3E5629401400985676585636CCA
:1015E900756D01C3E56278FA985021307404E52AD3
:1015F900601A78F0306B058567647820C3E54198F7
:101609005002A1140536E55F6002C118753600C2A3
:10161900AF120FD57887E6FE760211537887EEF67A
:10162900E4F522F523F524F525F526F568C268D2F7
:10163900AF12054A120FD5307406E52A700221F25D
:10164900788DE6C39401400241C661F1901A0D7884
:10165900201216D9E520B4A50CA31216D9E520B499
:101669005A03021677120FEA121697021696901A63
:101679000378807B0A1216D9A308DBF9901A0F7830
:101689008C7B181216D9A308DBF9901A2722C2AF4E
:101699001217181216F2901A00740E1216DEA3749D
:1016A900041216DEA374141216DE901A0378807BD6
:1016B9000A1216DDA308DBF9901A0F788C7B181231
:1016C90016DDA308DBF912172B121709901A272226
:1016D900E493F622E6438F01538FFD75EF0275B748
:1016E900A575B7F1F0538FFE22438F02438F017521
:1016F900EF0275B7A575B7F1901A0DF0538FFC225B
:10170900901A0D74A5D1DE901A0E745AD1DE227A80
:101719003079D07820901A40D1D9E520F709A3DA99
:10172900F7227A3079D0901A40E7D1DE09A3DAF9A5
:1017390022AB77A878BB01027980BB02027981BB11
:1017490003027982BB04027994BB05027983BB0643
:10175900027986BB07027992BB08027987BB090225
:10176900799CBB0A027988BB0B027989E8F7227C4C
:1017790005120563DCFB22C2AF12057312057A124A
:10178900058112058812055412057312057A12058E
:101799008112058812055412057312057A12058102
:1017A900120588D2AF22C2AF12058812058112052F
:1017B9007A12057312055412058812058112057AE9
:1017C90012057312055412058812058112057A1241
:1017D9000573D2AF22AE77AF78C2AF120573120587
:1017E90073120573120554DEF2120588120554DFCF
:1017F900F8D2AF22F1801217781217787577017530
:1018090078017579001217DE7C05AD5F120563C397
:10181900ED955F70F5C3E55F9401400AC3E55F94F8
:10182900FF403702184012173A121697121780C252
:10183900AF75EF12121778DCD10579C3E5799403F6
:10184900500280C11217780578E5771490009F93AC
:10185900F808C3E57898500280A81217781217780B
:0E1869000577C3E577940C50028094120FEAC5
:0B187700121697C2AF75EF121217781F
:0319FD0002115480
:101A00000E041407070104FFFF0A020101A55A0191
:101A100000B4FFFFFF03FF01FF25D078C804FF01DA
:081A200000FF0A010100FFFFB5
:101A400023526F746F724765656B73323041232088
:101A500023424C48454C4923463333302320202031
:101A60002020202020202020202020202020202076
:101C0000C2AFC2D353D9BF7581C043B20343FF8073
:101C1000752438752503B1C975EF0275E24043F1AB
:101C20002053A4DF75D400D2857DFA780379E67C51
:101C300010752200752300901DD67B0675249875BB
:101C400025013085028142208508D8FBD9F9DCF7CF
:101C500081B4308508D8FBD9F9DCF781B4B189E4C7
:101C600093A3C39A6004DDC381B4DBDBB17B600264
:101C7000812B7B08E493FAA3B15CDBF87A30B15C8A
:101C8000752200752300B17BEAFCEBFDC3ED94FEE9
:101C9000400EB17B8A278B28ED30E0048A828B834B
:101CA000B17B7AC270D8C3ED94FE601350CEBD00F4
:101CB00025EC60097520007521FF0200008100A855
:101CC00027A9280809D804D90281D3B17FEA89AAB3
:101CD000F281C50D81A0C3ED94035049EDA2E092BD
:101CE000007AC5C3E5829400E583941C50902000DF
:101CF00010438F02438F0175B7A575B7F1F030001F
:101D00001FA827A9280809438F01538FFDD804D99C
:101D100002A12089AAE275B7A575B7F1F0A3A10DBC
:101D2000538FFC817C7AC1BD030CE493A3FAB140CC
:101D3000DCF8B138817C817EAA22AB23B15CEBFA5E
:101D4000EA6222752608C3E52313F523E52213F57D
:101D50002250066323A0632201D526EAB1C9B1C986
:101D600075260AEAF4200102D285300102C285B14B
:101D7000C9C3134002C201D526EB22B17FEAFB2082
:101D80008502A17F308502A184752608AE24AF2587
:101D9000C3EF13FFEE13FEB1CDB1C9C3EA13308513
:101DA000024480FA30E703632201C3E52313F523DD
:101DB000E52213F52250066323A0632201D526D91C
:101DC000E52265236523F52222AE24AF250E0FDE22
:101DD000FEDFFCD20122424C48656C693437316326
:041DE000F3300601D5
:00000001FF
